:020000040000FA
:020000003F2B94
:08000800A000030EA10064003A
:100010001630810056206F20EC20210E8300A00EA8
:10002000200E0B110900FF30A800B630AB002530C0
:10003000AE002030B000B101B201B301B401B5018E
:10004000B601CA01CB01CC01CD01CE01CF01D00157
:10005000D101D201D3012511A5112513A601A616A0
:10006000F9210130D900DA000930DD000D30E0005F
:100070000330DE000800850107309F00031383165C
:10008000003085004030860003138312AC01AD01BF
:1000900008000B118B178B16810164000313831664
:1000A000D83081000313831281010800A51D6E283A
:1000B000251D6E28DB0B68288030DB00DA0B6828F2
:1000C0001030A506590859075907DA00DA03DA0390
:1000D000251E6E282D08803AAD0086000800A90A6A
:1000E0000319A80F7E28A514EF30A800FE30A90040
:1000F000AA0B7E28BC30A9002B08AA000800DE0845
:100100000319DF2837083102031D9A283808320204
:10011000031D9A2839083302031D9A283A0834022D
:10012000031D9A283B083502031D9A283C08360215
:100130000319B7283708BD003108B7003808BE00DA
:100140003208B8003908BF003308B9003A08C000C7
:100150003408BA003B08C1003508BB003C08C200A7
:100160003608BC006008E100E2005E08DF00E20B38
:10017000C1286008E200DF0BC1285E08DF00610BC8
:10018000E10061086202031CD2283708C300380866
:10019000C4003908C5003A08C6003B08C7003C083F
:1001A000C800EB283D08C3003E08C4003F08C50056
:1001B0004008C6004108C7004208C800EB283108C3
:1001C000C3003208C4003308C5003408C60035082F
:1001D000C7003608C80008002D088039AD00860029
:1001E000063032210830A2000310300C03182030F2
:1001F000B00030184308B018440830194508B01949
:100200004608301A4708B01A4808A202831C033E69
:10021000AC0085002D0880393004AD00A2002F0805
:100220003005031916292D088039AD00AE0B2D2994
:100230002530AE002208860000000608A2002D0826
:100240008600220840390319292922083F39D7049A
:100250002D292208FF3A3F39D7052D088600B01A0C
:100260007F200800A200A20B332908005708580677
:1002700003194B29A7015705D800D8194C21D818C4
:100280005621581A63215819702158187D21D81AFF
:100290008A215708D80008000310A60C0318522919
:1002A000F9215529A601A616F9210800A61A9721B9
:1002B000261A9E21A619A0212619DC21A618E321C1
:1002C0002618F8210800A61AC521261AB321A61956
:1002D000B5212619DE21A618EC212618F8210800E0
:1002E000A61AC821261ACF21A619CF212619CF2157
:1002F000A618CF212618F8210800A61AC521261A0B
:10030000D021A619D8212619E021A618BE21261829
:10031000F8210800A61AC521261AD321A619D3212F
:100320002619D321A618D3212618D3210800251178
:100330000830A5061030B606A512080013230800E1
:1003400052082723D200251CA82953083323D300A1
:100350005308023C031DB2295208043C031DB22974
:10036000D201D30108000923080050082723D00038
:10037000251CBD2951083323D1000800DE0A5E0880
:10038000093C03180800DE010800A5122511080029
:10039000251DCE292511A5165D08DC0008000800E2
:1003A000CA01CB0108002511A601A616F9210800F3
:1003B0005D082723DD000800AB030800AB0A080036
:1003C0004030A5060800A5151030B6042515D90B38
:1003D000EB290930D9000800A5151030B604251501
:1003E000D90A5908093C0318F729D901D90A080084
:1003F0000800EF30B105B205B305B405B5051030FE
:10040000261AB504A619B4042619B304A618B20412
:100410002618B1040800A61A1822261A1822A619AE
:10042000572226197122A618A5222618BC220800D8
:100430003108F0394A04B1003208F0394B04B200F7
:100440003308F0394C04B3003408F0394D04B400DB
:100450004E08A3004F08A400A61E492A251F492ABA
:10046000CF080319432ACF18392A4E08023C031833
:10047000492AA303A303A31F412A23080A3EA3007A
:10048000A403A403492ACE08031D492AA30AA30AE8
:10049000A40A3508F0392304B5003608F0392404DD
:1004A000B600B608031D552A562AAF0108000230CF
:1004B000AF003108F0395D04B1003208F039B20004
:1004C0003308F0395004B3003408F0395104B40053
:1004D0003508F0395204B5003608F0395304B60037
:1004E00008000830AF00D501D6012B08D4006430D5
:1004F000D60AD4020318782AD407D6030A30D50ABC
:10050000D40203187F2AD407D5033108F0395404E4
:10051000B1003208F0395504B2003308F0395604FE
:10052000B3003408F039B4000230251F0430A300B2
:100530003508F0392304B5000130251F0230A3002F
:100540003608F0392304B60008002430AF00310823
:10055000F0395904B1003208F039B2003308F039EB
:10056000B3003408F0395E04B4003508F039B50042
:100570003608F039B6000800AF013108F039B10093
:100580003208F039B2003308F039B3003408F039DA
:10059000B4003508F039B5003608F039B600080067
:1005A000CA08031DE92ACB08031DE92A4C0850029A
:1005B000031DE82A4D085102031DE82A4E08520285
:1005C000031DE82A4F085302031DE82A2515E92ACE
:1005D00025110800A51EF02ADC0BF02A2515A5120E
:1005E0000800A70A14302702031CF92AA601A61640
:1005F000F9210800A51C262BA510F1224A08272363
:10060000CA00251C252B4B083323CB00251C252B8A
:10061000EA224C082723CC00251C252B4D08332328
:10062000CD00251C252B4E082723CE00251C1B2B77
:100630004F082723CF004F08023C031D252B4E08EF
:10064000043C031D252BCE01CF01D022080025102C
:10065000C900490AC900093C0318312B0030251490
:10066000322B490808002510C900490AC900053C79
:1006700003183D2B003025143E2B49080800132099
:0C0680003B2049203621FA220B22422B9D
:02400E00053F6C
:00000001FF
